:10000000F2C300000DC4000025C4000009C40000B4
:1000100007C4000005C4000003C4000001C40000C0
:10002000FFC30000FDC300000C94F92DF9C30000CC
:10003000F7C30000F5C30000F3C30000F1C30000E4
:10004000EFC30000EDC30000EBC30000E9C30000F4
:10005000E7C30000000000000000000000000000F6
:100060000000000000000000000000000000000090
:1000700000000000000000007E0F00D4FFFFFFC75B
:100080000000007800000000000000002A2B28007B
:100090000000000000000000000000000000002937
:1000A000000000002C1E3420212224342627252E77
:1000B000362D3738271E1F202122232425263333AF
:1000C000362E37381F0405060708090A0B0C0D0EDB
:1000D0000F101112131415161718191A1B1C1D2FA7
:1000E0003130232D350405060708090A0B0C0D0EC7
:1000F0000F101112131415161718191A1B1C1D2F87
:100100003130354C05010980A101850319012AB759
:1001100000150126B700950175108100C0050C0976
:1001200001A101850419012AA002150126A002954A
:100130000175108100C00660FF0961A10109621507
:100140000026FF009520750881020963150026FF2F
:1001500000952075089102C005010906A101050757
:1001600019E029E71500250195087501810295011F
:10017000750881030507190029FF150026FF009562
:100180000675088100050819012905150025019546
:100190000575019102950175039103C01C0376005A
:1001A000690061006C003A006600360034006300AC
:1001B000320062003300630000000A035300500065
:1001C0003600340000000A0359004D0044004B0083
:1001D00000000403090409025B00030100A0FA09FE
:1001E0000400000103010100092101010001224472
:1001F0000007058103080001090401000203000053
:1002000000092101010001222200070584030800E2
:1002100001070504030800010904020001030000AE
:1002200000092101010001223200070583030800B3
:100230000112011001000000084D59645300020131
:1002400002030100000000000000000000000000A8
:10025000002C00E600E700500051004F003C000079
:1002600000E000E300E2002C002152230000001116
:10027000001000360037003800E50052000000E1B1
:10028000001D001B0006001900050000000B000DFA
:10029000000E000F00330034002800000039000475
:1002A000001600070009000A00000018000C0012E8
:1002B0000013002F003000310000002B0014001A42
:1002C0000008001500170000002400250026002764
:1002D000002D002E002A00000029001E001F002013
:1002E000002100220000001C0000000000000000AF
:1002F00000000000000000000000000000000000FE
:1003000000000000000100010001000100010001E7
:100310000001000000010001000100010001003F98
:1003200000000001000100010001000100010001C6
:1003300000000001000100010001000100010000B7
:1003400000010001000100010001000100010000A6
:100350000001000100010001000100010000000196
:100360000001000100010001000100010000000186
:1003700000010001000100010001000000400041F7
:100380000042004300440045000100000001003A23
:10039000003B003C003D003E00000001000000006A
:1003A000000000000000000000000000000000004D
:1003B0000000000000000000000100010001000139
:1003C0000001000100010000000100010001000126
:1003D0000001000100000001000100010001000116
:1003E0000001000100000001000100010001000106
:1003F00000010000000100010001000100010001F6
:1004000000010000000100010001000100010001E5
:1004100000000001000100010001000100010001D5
:1004200000000001000100010001000100010000C6
:1004300000010001000100010001000100010000B5
:1004400000010001000100010001000100000001A5
:10045000000000000000000000000000000000227A
:1004600023252628292A2C2D2F3032333536383AA9
:100470003B3D3E4042434547494A4C4E50515355FF
:1004800057595A5C5E6062646668696B6D6F717320
:100490007577797B7D7F81838587898A8C8E909221
:1004A0009496989A9C9E9FA1A3A5A7A8AAACAEAF2C
:1004B000B1B3B4B6B8B9BBBCBEBFC1C2C3C5C6C771
:1004C000C9CACBCCCDCED0D1D2D2D3D4D5D6D7D722
:1004D000D8D9D9DADADBDBDBDCDCDCDCDCDDDDDD6A
:1004E000DDDCDCDCDCDCDBDBDBDADAD9D9D8D7D766
:1004F000D6D5D4D3D2D2D1D0CECDCCCBCAC9C7C613
:10050000C5C3C2C1BFBEBCBBB9B8B6B4B3B1AFAE50
:10051000ACAAA8A7A5A3A19F9E9C9A9896949290F6
:100520008E8C8A89878583817F7D7B7977757371CE
:100530006F6D6B6968666462605E5C5A59575553AB
:1005400051504E4C4A4947454342403E3D3B3A3864
:1005500036353332302F2D2C2A292826252322FF09
:10056000AA7F5540000101010101010101010202C0
:100570000202020202020203030303030303030451
:10058000040404040404050505050506060606061C
:10059000070707070708080808090909090A0A0AD6
:1005A0000B0B0B0C0C0C0D0D0D0E0E0E0F0F0F1078
:1005B0001011111112121313141415151616171702
:1005C000181819191A1A1B1B1C1D1D1E1E1F20206E
:1005D000212222232424252626272829292A2B2CB8
:1005E0002D2D2E2F30313232333435363738393ADB
:1005F0003B3C3D3E3F404142434445464748494AD3
:100600004C4D4E4F50515354555658595A5B5D5EA0
:100610005F616264656668696B6C6D6F707273753B
:1006200077787A7B7D7E8082838587888A8C8E8F9F
:1006300091939596989A9C9EA0A2A3A5A7A9ABADCD
:10064000AFB1B3B5B7BABCBEC0C2C4C6C9CBCDCFBB
:10065000D1D4D6D8DBDDDFE2E4E7E9EBEEF0F3F569
:10066000F8FAFDFF1E0F0500047F3F1F643214647B
:100670003214783C1E1E140A05FD377A585A0000C1
:1006800004E6D6B4460200210116000000742FE5EE
:10069000A3E002F401295D003D8889C65436C317E2
:1006A0004FE4E621D90942F33DA3924D5DE896ADB2
:1006B0003D1C694D102E8CA62813C8A825474BFA5F
:1006C000CFB3B0E4382A0942B5B834C5F0EA074BD5
:1006D0005E7732E5710B8DA6C1C0CE0EA182F261AC
:1006E000B1E53991BBF0DA9A1FE9D6CC9DD20195DC
:1006F000DF935C8D33881AD1531EAC768D32E97B43
:10070000514FEAE24245171A7249FAF78D6C24A656
:10071000BF0901B8CCBBF8513E0C5FB0389981518C
:100720003E5903714AF28552E85E24A35D5288E780
:100730000707A74C82FF21B8B678E8F33B9C94C02A
:100740005F08C6C295DB8430FF6EEDAD353F0274A5
:100750004E55E25A35461A1F5CE7BEF09B2C5019E5
:1007600007B99720D209E8677D943114095BDC71E1
:10077000129B33CC7F6E1150332851A15EC1EF73B1
:10078000AFDEDC69D6F3684982D0111B10E9B19362
:1007900043E25DC4F737EA6B8DF503C1E5B3E229A7
:1007A000EF0F9A7568D5956A0A7E840BB5E14D44C2
:1007B000C1E912020835CB80339E622FD89333FAF9
:1007C0000700000000796DEB0DE09AE4150001C50B
:1007D00002F5050000C42CC34FB1C467FB02000042
:1007E000000004595A0011241FBECFE5D8E0DEBF37
:1007F000CDBF24E0A8E2B1E001C01D92AC38B20741
:10080000E1F711E0A0E6B0E0E6E1F4E602C0059011
:100810000D92A832B107D9F70E94EB260C94A831AB
:10082000EFCBA82FB92F80E090E041E050EA60952F
:1008300030E009C02D9182279795879510F0842785
:100840009527305EC8F36F5FA8F30895EADF8D93B4
:100850009D930895CF93CFB7CF93C395839BE9F72B
:10086000839B0EC0839B0CC0839B0AC0839B08C0E4
:10087000839B06C0C0916604C395C0936604A6C05E
:10088000DF93C0916504DD27C659DB4F839B02C00F
:10089000DF91E6CF2F930F931F9300B32FEF03FB4E
:1008A00020F94F933F9310B34FEF012703FB21F93A
:1008B0003BE031C04E7F012F10B3216028C0102FC4
:1008C0004D7F2260000000B329C04B7F2460012FC0
:1008D000000010B32BC010B3477F28602AC04F7EA2
:1008E00000B320612CC04F7D10B320622FC04F7B1E
:1008F00000B3206432C0422700B349934FEF000099
:10090000102713FB20F910B31C70C9F1297F91F255
:10091000012703FB21F900B3237F89F2315058F1FD
:10092000102713FB22F910B3277E79F2012703FB6E
:1009300023F92F7C81F200B3102713FB24F92F79C0
:1009400071F200C010B3012703FB25F92F7359F290
:1009500000C000B3102713FB26F9223040F200C07C
:1009600010B3012703FB27F9243028F64F772068BE
:1009700010B30000F9CF10E81ABF00271CC03B508D
:100980003195C31BD04010E81ABF0881033C11F118
:100990000B3401F1209163041981110F1213EDCF73
:1009A0004A81441F093669F10D3211F0013E29F7E1
:1009B0004F7009F0042F009369043F914F911F91EC
:1009C0000F912F91DF91CAB7C7FD47CFCF91CFBF0E
:1009D000CF91189520916904222379F3109167042F
:1009E000112309F044C034300AF443C03093670443
:1009F00020936404109165043BE0311B309365043F
:100A000038C000916704013094F50AE54F7049F44D
:100A10003091650034FD2FC000936500C0E4D4E040
:100A20002EC0433059F0443091F030914B0434FDE6
:100A300022C000934B04CCE4D4E021C03091800468
:100A400034FD19C000938004C1E8D4E018C030918F
:100A5000570434FD10C000935704C8E5D4E00FC01C
:100A60002795A8F45150A9F4220F0000F9CF4AE5C8
:100A700003C042ED01C0432FC4E1D0E032E011B326
:100A80001C60939A11BB02B320E41CE05F93012722
:100A900056E002BB279520F4515021F4220FF9CFE4
:100AA000012756E000003B5A02BBD0F2279528F4FC
:100AB000515029F4220F0000F9CF012756E0279565
:100AC00002BB20F4515021F4220FF9CF012756E048
:100AD0002991332302BB21F6037F10916804110F83
:100AE000C651D04002BB11F01093630410E81ABF46
:100AF000086011B3137F402F437F5F9100C000C097
:100B000002BB11BB42BB59CF9C01FB019A958115D9
:100B10009F4120F5832F8170B32FB270AA27732FC6
:100B200074706627532F5870442734FF0DC0829588
:100B3000807FAB2B09F08062672B09F08064452B26
:100B400009F0806809950895AB2B09F08260672B46
:100B500009F08460452BB1F38860F4CF80E0F2CFD8
:100B6000982F92959F7024E0911102C020E0982F59
:100B7000892F86958695811511F02E5F982F892FE4
:100B80008695820F089580FF08C0909A81FF07C064
:100B9000919A82FF06C0969A08959098F7CF9198FF
:100BA000F8CF9698089580933B04089580933C0471
:100BB000089521E030E001C0220F8A95EAF7809184
:100BC0003C04822BF3CF21E030E0A90102C0440FA6
:100BD000551F8A95E2F7CA01809590913C048923BC
:100BE000E5CF292F963090F58F3080F590E03FE0EB
:100BF000239F800D911D1124282F277041E001C0F3
:100C0000440F2A95EAF723E0969587952A95E1F710
:100C1000FC01EE0FFF1FE80FF91FE054FD4F20E02D
:100C200030E070E05191DF01CB01022E02C09695B9
:100C300087950A94E2F7817081958527842385271B
:100C40008E932F5F3F4F2330310561F70895292F91
:100C5000963078F58F3068F590E03FE0239F800D67
:100C6000911D1124682F677023E0969587952A952A
:100C7000E1F7FC01EE0FFF1FE80FF91FE054FD4FF5
:100C800040E050E080E0219130E0062E02C0369531
:100C900027950A94E2F721703327042E01C0220F12
:100CA0000A94EAF7822B4F5F5F4F4330510559F7A3
:100CB000089580E0089590913C0421E030E0F9012E
:100CC00001C0EE0F8A95EAF7D90102C0AA0FBB1F37
:100CD0006A95E2F7EA2B01C0220F4A95EAF7892FBD
:100CE0008E23E81303C0892F822B60CF2095822F9B
:100CF0008923FBCF80916E0290916D02981301C001
:100D000008958F5F8770FACF90918703809589232C
:100D100080938703282F2770211110C0891771F045
:100D200090913E0492FF0AC08695869586954BDF8A
:100D3000109287031092890310928803089590916E
:100D40008403982B909384030895982F9095809115
:100D500084038923809384030895809183038115FC
:100D600031F01092830310928B0310928A0308953E
:100D7000803E9105D9F1C8F48133910509F482C010
:100D800048F48932910509F472C08A32910509F458
:100D900080C0089589339105E9F082389105D1F03A
:100DA0008533910509F45EC00895843E9105D9F11B
:100DB00048F4823E910539F1833E910549F181EE77
:100DC00090E00895863E9105C9F1873E910509F4AA
:100DD0003EC0089520913D042370211164C02091EC
:100DE0003E0423FF14C089E290E0089520913D0461
:100DF00020FD45C030913E0430FF09C024FD24C0D1
:100E000083EE90E0089520913D0422FDF7CF0895F0
:100E100020913D0422FD44C030913E0430FD43C08A
:100E200024FFF5CF11C020913E0421FFF0CF809127
:100E30003D0484FD09C087EE90E0089520913D04B3
:100E400023FFE5CF24FFF7CF80E090E008952091C5
:100E50003D0423FD2BC030913E0431FFE1CF84EEF1
:100E600090E0089520913D0425FFD1CFBCCF209183
:100E70003D0425FD1EC020913E0423FFC8CF89E319
:100E800090E0089520913D0426FFC1CF8AE290E0D2
:100E9000089520913D0426FFBACF81E390E00895A4
:100EA00082EE90E0089580EE90E0089586EE90E066
:100EB000089585E390E0089590913D0492FF10C05D
:100EC00041E0282F2471243009F040E031E0282F40
:100ED0002871283009F030E0431711F02CE0822708
:100EE00093FF10C041E0282F2471243109F040E025
:100EF00031E0282F2871283109F030E0431711F034
:100F00002CE0822730913E0430FF10C051E0282FA2
:100F10002171213009F050E041E0282F287128305C
:100F200009F040E0541711F029E0822731FF10C08A
:100F300041E0282F2171213109F040E031E0282FD4
:100F40002871283109F030E0431711F029E0822799
:100F500094FD877E08951F93CF93DF9309DFEC0103
:100F6000811522E5920708F052C0811540E59407EB
:100F700008F0CDC0803E910520F58D3C910508F02C
:100F8000A1C0883A910570F4853A910508F097C0A0
:100F900081309105B9F10497813A910598F1C0E04B
:100FA000D0E030C0885A91094B97C8F7C85AD0E0B2
:100FB000CC0FDD1FC554DF4F0990D881C02DD464FC
:100FC00021C0811550E49507B0F4C11580E2D8071F
:100FD00008F0B3C0C83ED105A8F0CE019A9581159E
:100FE0009F41E8F68D2F68DF182FCE019927C0DECC
:100FF000EC01D12B07C09927BBDECC27DF70C82BB3
:10100000D92BD06ACE01DF91CF911F9108958038FE
:1010100042E59407C8F5803652E5950708F05BC0B5
:10102000C03482E5D807D0F4C03292E5D90708F081
:101030004BC08C2F8695869520E2829FC00111249B
:10104000C37021E030E0A90102C0440F551FCA95CA
:10105000E2F7EA01C82BD92BDD68D4CF8C2F869517
:101060008695877050E2859FC0011124C37021E0EE
:1010700030E0A90102C0440F551FCA95E2F7EA010A
:10108000C82BD92BDC68BECF803C52E5950758F4BD
:101090008F71C03AD245A0F590E0982F8827EC01D7
:1010A000C46FD06AAFCF805C9245809708F077CF4D
:1010B000DC2FCC27CC27DF71C06FD06AA3CFA497D9
:1010C000D064A0CFD0659ECFCF71D0E0DC2FCC27ED
:1010D000C16FD06A97CF86958695877020E2829FF0
:1010E000C0011124C37021E030E0A90102C0440F07
:1010F000551FCA95E2F7EA01C82BD92BDA6882CFCF
:10110000DBDEC82FD0E0DC2FCC27D0627BCF8F7105
:10111000D3DE93E0CC0FDD1F9A95E1F7CC27DF708B
:10112000282F30E084FF05C050E1859F90011124F5
:101130003327C22BD32BD06965CF8D2F8F71BCDEA7
:10114000182FCE01992714DEEC01D12BDECF80E0E1
:1011500008950895CF92DF92EF92FF921F93CF935D
:10116000DF93172FE82FF0E0EC59FA4F71110CC004
:10117000E4918E2F7E2F6E2FDF91CF911F91FF90E4
:10118000EF90DF90CF900895E62EF12CC72ED12C52
:10119000F491EF2F86E0689F90011124CFEFD0E00B
:1011A000C901BE010E94A22FAB01EE0CFF1C65E538
:1011B000649FC001659F900D1124E81AF90A6E2DF5
:1011C000660F6E0D7E01EC18FD08FE9DD001FF9D9F
:1011D000B00D11248B2F169F70011124EF2CFF24CA
:1011E0006E01CE18DF087601FE9D6001FF9DD00CD8
:1011F00011247E01E61AF108B701169F7001179FAE
:10120000F00C1124EF2CFF24CE19DF09FC9F700194
:10121000FD9FF00C11247F2D43305105C1F02C3F70
:10122000334058F441305105B1F04230510509F0D6
:10123000A2CFEB2F8F2D7F2F9ECF4430510571F021
:101240004630510509F497CF7B2F8D2D94CF7D2DFE
:10125000EB2F8F2F90CF7F2FED2D8DCFEF2D7B2F6D
:10126000F8CFCF93982F762F842FC22F692F72DF5C
:10127000472F282F8C2F90E049D2CF91089580914D
:101280007A03843060F48370846080937A03809161
:101290007D038B3F18F08AEF80937D0308958C3A8D
:1012A000B0F38370886AF1CFCF93DF9380917A0394
:1012B00080FD0BC0C0E0D0E020E040E060E0CE0167
:1012C00025D22196CC30D105B9F7DAD3DF91CF9171
:1012D0000895FF920F931F93CF93DF93182F062F3C
:1012E000F42E80917A0380FF0CC0C0E0D0E02F2D57
:1012F000402F612FCE010AD22196CC30D105B9F70B
:10130000D3DFCDB7DEB7E5E00C94DF2FCF93DF93CB
:10131000EC0120917D039C81892F817090FD822FAB
:10132000692F627091FD622F492F447092FD422F08
:10133000D0DF8C8190E00196877099278C83DF91B4
:10134000CF910895982F762F842F20917A0320FF34
:101350000AC04B3F08F08AEF692FFCDE962F672FFB
:10136000482F892FB6CF0895CF93DF93EC01EAE79A
:10137000F3E0438162818C81E5DF8C818F5F8C8318
:10138000DF91CF910895CF93DF93EC01EC81F0E0F2
:10139000E15AFB4F4491EAE7F3E062818181D2DFB9
:1013A0008C818F5F8C83DF91CF910895FF920F9393
:1013B0001F93CF93DF93EC01F12C00E010E04091FC
:1013C0007D034B3F08F04AEF8C81980160917C03CC
:1013D0008F0D47DF0F5F1F4F85E1F80E0C301105B1
:1013E00071F762DF8C819A8190FF07C08F5F8C83D9
:1013F000CDB7DEB7E5E00C94DF2F8150F8CFEF9248
:10140000FF920F931F93CF93DF93FC018281FF2400
:10141000F39480FF02C0FF24FA94C0E0D0E020E003
:1014200040E060E0CE0172D104E010E0E12C809158
:101430000A028E0D8D30A4F16CE00E94F92F892FE5
:10144000082E001C00088C170D0691F440917D03B6
:101450000403A001112455954795559547954B3F99
:1014600008F04AEF9E0160917C0380917B03F9DED6
:10147000EF0C01501040D9F62196CC30D10579F609
:1014800013DF80910A02F1E0FF120EC0811591F086
:10149000815080930A02CDB7DEB7E6E00C94DE2FD0
:1014A00087FFCECF845FCCCF90E00196BE010E9433
:1014B0000630EFCF8BE0EDCFCF93DF93C0E0D0E0ED
:1014C00020E040E060E0CE0121D12196CC30D10572
:1014D000B9F7C0E0D0E080910902082E001C000896
:1014E000C817D00574F180916C00082E001C00080C
:1014F0008C170D0634F140917D034B3F08F04AEF05
:101500009E0160917C0380917B03ABDE2196CC3001
:10151000D10509F7C9DE80916B0090910902980FFF
:101520009093090220916C00280F20936C001216F2
:1015300014F49B301CF0819580936B00DF91CF9168
:10154000089520E040E060E0CE01E0D0DFCFA6E0EB
:10155000B0E0EDEAFAE00C94C02F8D839E83AD815C
:10156000BE811496FC912F2F30E0D9010E94993151
:101570009B01AC010E9467316B017C0180E290E02D
:101580009C012F1B3109F901A5E5B0E0A7019601E7
:101590000E94673169837A838B839C839F01DF017B
:1015A0000E9426309B010E942C309B01AC012C0D27
:1015B0003D1D4E1D5F1D69817A818B819C810E943A
:1015C0007731022F30E00A32B8F5C901880F991F30
:1015D000820F931F95958795182F1095E12CF12C6C
:1015E00085E5D82ED01A8D2DE1FC802F412F1B3F91
:1015F00008F04AEF970160917C0333DE5FEFE51A54
:10160000F50A8CE0E816F10471F74EDEAD81BE817B
:1016100014969C9181E0911519F0903219F48FEF96
:1016200080936A0080916A00890FED81FE81848336
:101630002696E8E00C94DC2F85E590E0AC01421B97
:10164000530B9A01CA01880F991F820F931F97FFAE
:10165000C1CF0196BFCF0F931F93CF93DF93EC01C0
:1016600020E030E060917C0380917B039C818901C4
:101670000F5F1F4F2630310554F4911501F1409151
:101680007D034B3F08F04AEFECDD9801EBCF911161
:1016900016C040917D034B3F08F04AEFE2DD980110
:1016A0000C301105F9F600DE8C8190E00196817016
:1016B00099278C83DF91CF911F910F91089540E07E
:1016C000EDCF81152CE7920741F420914102309132
:1016D0004202232B11F480E090E00895E2EFF2E063
:1016E00080E090E066E675E249E855E22BEF35E2EE
:1016F00077836683518740873387228797878687DA
:10170000019670968830910599F70895FC01EE0FC7
:10171000FF1FE80FF91FEF5AFE4F618340832283BA
:1017200008951092CD031092CC03ECE8F3E085818C
:10173000811102C014821682379683E0E43CF807D8
:10174000B1F70895AC013091CF036091CE03232F00
:10175000621301C00895822F90E0FC01EE0FFF1F7D
:10176000EC53FC4F0190F081E02DE417F50791F464
:1017700067E0649FF001659FF00D1124E457FC4F72
:1017800041E044832313E6CF019683709927809329
:10179000CF0308950196282F2370DACF0F931F935C
:1017A000CF9301E010E0082E01C0000F0A94EAF781
:1017B000C09182039C2F9023911115C090918703B3
:1017C000969596959695891306C010928703109268
:1017D000890310928803EDD9C027C0938203CF916B
:1017E0001F910F910895EFD9F7CFFA01309709F0C3
:1017F00009950895E0916B02F0916C02309739F0F1
:101800000190F081E02D309711F00995089580E066
:101810000895A3E0B0E0EFE0FCE00C94C62F9C013B
:1018200080914E0190914F0182179307B1F0309350
:101830004F0120934E01E0916B02F0916C023097C2
:1018400061F00084F185E02D309739F083E08983E1
:101850003B832A83CE01019609952396E2E00C94FE
:10186000E22FA3E0B0E0E7E3FCE00C94C62F9C017C
:1018700080914C0190914D0182179307B1F0309304
:101880004D0120934C01E0916B02F0916C02309776
:1018900061F00084F185E02D309739F084E0898390
:1018A0003B832A83CE01019609952396E2E00C94AE
:1018B000E22F9C01FC0132968FEF90E04191461798
:1018C00051F08F3F19F4411101C0892F9F5F96306D
:1018D000A9F78F3F09F40895280F311D87FD3A9528
:1018E000F901628308959C01FC013296285F3F4F05
:1018F0008191861302C0DF011E92E217F307C1F740
:1019000008958091670008952FB7F8946091480179
:101910007091490180914A0190914B012FBF089528
:1019200008950895FC018381833081F130F4813082
:10193000E9F0823019F180E00895813209F449C05C
:101940008232C9F7248135812130310509F45AC02A
:101950002230310509F45DC0232B69F788E591E059
:1019600090933F0180933E0184E4089581E392E0E7
:1019700090933F0180933E0182E1089586ED91E0CE
:1019800090933F0180933E018BE5089582818230E0
:10199000E9F050F4811112C082ED91E090933F0183
:1019A00080933E0184E00895833029F68CE991E02C
:1019B00090933F0180933E018CE1089586EC91E085
:1019C00090933F0180933E018AE008958AEB91E075
:1019D000F7CF848195818130910571F08230910536
:1019E00071F0892B09F0A7CF88EE91E090933F0129
:1019F00080933E0189E0089581E092E0F7CF81E293
:101A000092E0F4CF26E331E030933F0120933E0192
:101A1000089584E091E090933F0180933E0182E33A
:101A20000895E0916B02F0916C02309749F00284C6
:101A3000F385E02D309721F060E283E492E0099590
:101A40000895E0916E0290916D0229E0E91302C0C1
:101A500080E00895AE2FB0E02E9FF0011124E159EF
:101A6000FD4F3181361306C03081381303C03581F4
:101A7000341304C0FD013196E770E8CF81E008958A
:101A800024E630E044E250E061E571E080EB0C9444
:101A9000E82EA3E0B0E0EFE4FDE00C94C52F8FEF5B
:101AA0009FEF909386008093850080913F04811181
:101AB0000EC00E94682E81E080933F042FEF8EE9D4
:101AC00094E2215080409040E1F700C0000019826C
:101AD0001A821FEF1B8324E630E043E050E0BE0192
:101AE0006F5F7F4F80E40E94E82E9C0190938600F8
:101AF00080938500892B41F58CE089831A821B83B2
:101B000024E630E043E050E0BE016F5F7F4F80E4A9
:101B10000E94E82E9C019093860080938500892B7B
:101B200099F484E189831A831B8324E630E043E03F
:101B300050E0BE016F5F7F4F80E40E94E82E9C0161
:101B40009093860080938500822F2396E3E00C9487
:101B5000E12F0C94682E089590913E0492FB222769
:101B600020F9281771F080FB92F990933E04609160
:101B70003D0470913E0484E090E00E94313182E0A7
:101B8000C3C808951F93CF93DF93962F122F632F0F
:101B90008430D8F49630C8F44F30B8F4C42FD0E075
:101BA000CC0FDD1F2EE1929FC00DD11D112494EBAF
:101BB000899FC00DD11D1124CE0189960E94183134
:101BC000612FCE018A960E941831DF91CF911F912B
:101BD00008950F931F93CF93DF93843030F56630D1
:101BE00020F54F3010F5C42FD0E0CC0FDD1F2EE1D3
:101BF000629FC00DD11D112434EB839FC00DD11DF8
:101C00001124CE0189960E94F730082F10E0102F82
:101C10000027CE018A960E94F7309801282BC9012F
:101C2000DF91CF911F910F91089580E090E0F8CF60
:101C3000462F672F2091670230916802232B81F491
:101C4000703F39F4403F61F48091650290916602E3
:101C50000895763028F44F3018F4843008F4B9CF62
:101C600080E090E00895A0E0B0E0E9E3FEE00C94AD
:101C7000C12F7C0100913C0480913B04082BC3E000
:101C8000D0E010E0C8010C2E02C0959587950A940B
:101C9000E2F780FD09C02197A8F7D12C8D2DCDB793
:101CA000DEB7E7E00C94DD2FDC2EB7018C2FC0DF10
:101CB00052D9019781F3F2CF0F931F93CF93FC0179
:101CC00087819085009789F4858100811181811534
:101CD00081F0611571F0C801C6DFC82F682FC801F7
:101CE0000E94F105B8018C2FA3DFCF911F910F91B6
:101CF0000895C8010E942706C82FF4CFCF93DF9321
:101D0000D82FC92FB0DF6D2F7C2F92DF24D9DF9120
:101D1000CF910895FC0184818115A9F08781908578
:101D2000009799F018D9282F92959F709630B9F0A6
:101D300080F4925F9F70923030F4203FD1F058F4DD
:101D400081E0283E58F080E0089580819181D6DFBF
:101D5000EACF9A5FEFCF81E0243FA9F7089591E0A1
:101D6000813F09F090E081E0283E08F080E0892B77
:101D7000089581E00895382F292FCB01A32FB22F8A
:101D800087369105A105B10520F487569C4F0C9428
:101D9000F73080E0089585E290E00E94F7308B37BD
:101DA00089F486E290E00E94F730803659F487E2A9
:101DB00090E00E94F73091E08F3B09F090E0892F8E
:101DC0008170089580E0FCCFAAE0B0E0EAEEFEE08A
:101DD0000C94BB2FC0904102D090420281E090E071
:101DE0009093420280934102812C912C10E0540187
:101DF00000E019C021E030E0133021F0F7018591B7
:101E000095919C01472D602F812FBCDE739422E0B9
:101E1000E20EF11C3FE07312EDCF0F5F8FE0A80ED2
:101E2000B11C063049F0C501880F991FFC01ED5B1C
:101E3000FD4F7F01712CDECF1F5FFAE58F0E911CE5
:101E40001430A9F61A8219821C821B821E821D82FE
:101E500018861F8288EC90E09A87898709EF12E044
:101E60009E012F5F3F4F79014AE050E0B801C70162
:101E70000E943531065F1F4F5701093433E01307C5
:101E800099F78AE0F70111928A95E9F74AE050E064
:101E9000B801C5010E943531065F1F4F0939F3E0D3
:101EA0001F07A1F7D0924202C09241022A96EDE0AC
:101EB0000C94D72FAAE0B0E0E0E6FFE00C94C02F2E
:101EC000E5E7F1E080E5DF011D928A95E9F7ECE8AE
:101ED000F3E088E3DF011D928A95E9F785E7C82ED4
:101EE00081E0D82E7F0109E413E0F701D182C0829E
:101EF0004AE050E0B801CE0101960E94E73088E048
:101F0000FE013196D60101900D928A95E1F78985FF
:101F10009A85D70113969C938E931297BAE0CB0EB5
:101F2000D11CE7E0EE0EF11C065F1F4F0939F3E00C
:101F30001F07D9F62A96E8E00C94DC2F282FCB0156
:101F4000283070F44AE0249F90011124B9016750B1
:101F50007D4F4AE050E00E94E73080E090E0089535
:101F60008FEF9FEF0895AAE0B0E0E9EBFFE00C945B
:101F7000C62F9C0197558115914068F4BE016F5F93
:101F80007F4F822FDBDF892B31F489859A852A9652
:101F9000E2E00C94E22F88EC90E0F9CFA0E0B0E012
:101FA000E4EDFFE00C94BA2FFC018280648081E0B4
:101FB0008483EFE5F4E09490EEEDF4E0E491009199
:101FC0007D030695015810E0000F111F012F112706
:101FD000CDECD1E0C12CD12CAA24AA94B12C772429
:101FE0007A94E919EE2EF12C83E0881630F4809172
:101FF0007B03888380917C038983611018C01B82D6
:102000001A824A814B3F08F04AEF96016981888124
:1020100028D98FEFC81AD80A25968CE0C816D104A3
:1020200019F742D9CDB7DEB7EEE00C94D62F8B81ED
:102030008115E9F081508B83789EC00111246C8159
:1020400070E00E94A22FFB01FF27E15AFB4F849111
:10205000E82FE9197E9EC0011124B7010E94A22F2A
:1020600080917D03689FB00111247A83CACF0E94BA
:10207000AF30B5010E940630801791070CF0C1CF38
:1020800083E0881688F00E94AF30B5010E940630C8
:1020900088830E94AF3020917C032695622F70E0E8
:1020A0000E940630280F29831A8280917D03893C83
:1020B00020F088EC8C838B83A4CF8431D8F784E123
:1020C000F9CF0F93CF93DF93CAE7D3E048815981CB
:1020D0006A817B8188E090E00E94293128813981E2
:1020E0004A815B816C817D818E819F8100E20E94AB
:1020F0004D30622F83E290E00E941831DF91CF9142
:102100000F910895EAE7F3E085E0808311828FEF75
:1021100082838AEF83831482CF01D3CF80917E03A1
:10212000833018F48F5F80937E038AE793E0C9CFF2
:1021300080917E03811519F0815080937E038AE798
:1021400093E0BFCFA0E0B0E0E8EAF0E10C94BB2F51
:10215000082FF62E142FE22E90917A0390FF25C0BF
:10216000E92FE695E695AE2FB0E0A057BF4F8C91D2
:10217000809378039C7F9430E9F4842F4B3F08F0E0
:102180008AEF602F7F2D0E94AA08962F672F482F75
:10219000892F9FD800937B03F0927C0310937D03DB
:1021A000E11419F08AE793E08CDFCDB7DEB7EDE0FC
:1021B0000C94D72F823019F410917D03EBCF863029
:1021C00019F400917B03E6CF8930D9F3893111F7F7
:1021D000E9518E2F8170782EE695F0E0E15AFA4FA2
:1021E000E491CE2FD0E0A12CB12CC12CD12C8CE0CD
:1021F000882E912CC501B4010E94A22F802F71104E
:1022000013C0860F412F1B3F08F04AEF96016F2D38
:1022100028D88FEFC81AD80AAC0EBD1E8CE0C8169D
:10222000D10441F741D8B6CF861BECCFEAE7F3E003
:10223000818121E043816281885F84CFEAE7F3E016
:10224000818121E04381628188507CCFEAE7F3E01D
:10225000628128E0620F08F46FEF21E04381818101
:1022600071CFEAE7F3E0628128E0621B08F460E0E6
:1022700021E04381818166CFEAE7F3E0438128E0F2
:10228000420F08F44FEF21E0628181815BCFEAE7E2
:10229000F3E0438128E0421B08F440E021E0628142
:1022A000818150CFA0E1B0E0E8E5F1E10C94B82FD6
:1022B000FE01319680E1DF011D928A95E9F707E082
:1022C00010E099E9A92E93E0B92E27E6422E512C71
:1022D000612C712C4F0173016201B1E14B16510465
:1022E000610471041CF080E1C82ED12CA601B50157
:1022F000C4010E940931AC0CBD1C0D2C000CEE0871
:10230000FF084C185D086E087F080150104019F74F
:102310006096E0E10C94D42F6FEF85E290E00E948C
:1023200018316FEF86E290E00E9418316FEF87E27C
:1023300090E00E94183160E088E290E00E9418313D
:1023400043DDB0DF6BE785E290E00E94183160E684
:1023500086E290E00E9418316FEB87E290E00C94E7
:10236000183160E081E090E00E943E3188E19CE01D
:102370000FB6F894A89581BD0FBE91BDFFCF1F93F6
:10238000CF93DF93782F162FEA01888184FF1EC038
:10239000898128E882278983AE014E5F5F4FFA0169
:1023A000272F392F710FD9012F5F3F4F8C918193C8
:1023B000872F821B1816BCF3612FCA010E942604C6
:1023C0001C5F1883DF91CF911F9108958AE5888360
:1023D000E3CFCF93DF9390916704935097FD14C0A0
:1023E00080916504CCE0D0E0C81BD109C659DB4F11
:1023F00080916404803108F06BC0983009F455C0B6
:1024000010926302109267048091650084FF3FC0C0
:10241000809164008F3FD9F1C82F893008F0C8E05F
:10242000982F9C1B909364009091400428E8922779
:10243000909340048115E9F080913E0190913F0115
:1024400020913D0126FF17C1FC012C2F41E454E0EF
:102450003491DA013C934F5F5F4F31962A95C1F773
:1024600001962FEF2C0F820F911D90933F018093C7
:102470003E016C2F81E494E00E94260484E08C0FDE
:10248000C83019F09FEF909364008093650084E159
:1024900090B39C70911106C08A95D1F71092680490
:1024A00010926304DF91CF91089580916302893186
:1024B00008F0A6CFA82FB0E0AD5BBD4F98E0FE01BD
:1024C00001900D929A95E1F7885F809363029ACF0D
:1024D0008D3209F0B4C0983009F094CF83EC80932A
:1024E00040048AE58093650010923D012881822F87
:1024F0008076811509F464C0803259F4898189306D
:1025000009F43FC040F4823049F1833099F18130C1
:1025100099F090E01BC08A3009F44EC08B30C9F7A7
:102520008C819D81892BA9F781E09A81911101C04D
:1025300080E080936800EDCF2C813D81232B49F70B
:1025400020E431E030933F0120933E018F818111DF
:1025500030C08E81891768F5982F2BC08091660056
:102560008093390189E391E090933F0180933E018C
:1025700091E0ECCF809168008093380188E391E08E
:10258000F3CF8A819B818115924069F48C819D8172
:10259000892B49F481E080933C018E819F81909347
:1025A0003B0180933A019FEF27FD9E8180E8809355
:1025B0003D019093640026CF8B8180936600A9CF64
:1025C0009A8110924904E981EC30A8F4F0E0E655D4
:1025D000FE4C0C94193024E632E081E005C01092E4
:1025E0004A0429E434E082E030933F0120933E0125
:1025F00016C09093680429E434E0F6CF9B819130B3
:1026000019F4CE018FD908C09230D9F39330C9F3B1
:102610009132B9F39232A9F390E490933D01982F4F
:1026200095CF90936402E7CF9BE490934C049093F2
:10263000810490935804DFCF29E434E0CECF809119
:102640003D0187FFDFCE80913A0190913B01892BBC
:1026500071F080913C01813051F488818093670052
:1026600010923B0110923A0110926400CBCE8EE1A1
:1026700080936500C7CEDC012C2F41E454E0FA01C1
:102680003D9130834F5F5F4F2A95C9F7E9CEFF92A6
:102690000F931F93CF93DF93082FD62F172FC42F9D
:1026A00085E0F82E033089F00430B1F080914B04BE
:1026B00084FF19C04BE454E06C2F8D2F912F5FDE07
:1026C000CDB7DEB7E5E00C94DF2F8091800484FF66
:1026D0000AC040E854E0F0CF8091570484FF03C063
:1026E00047E554E0E9CF75DE87E99AE30197F1F712
:1026F00000C00000FA94B1F6E3CFA0E0B0E0E3E858
:10270000F3E10C94BD2FF82EEB018A016A0193E0EE
:10271000D694C7949A95E1F79C2C5B01E12CE910C3
:1027200014C00770011561F083E0CC0CDD1C8A95A4
:10273000E1F7BE016C0D7D1D43E050E08F2DA7DF5A
:10274000CDB7DEB7EBE00C94D92F48E050E0B501EF
:102750008F2D9DDF88E0A80EB11CE394E0CF792F88
:10276000603229F440E250E0682F84E0C6CF08953B
:10277000CF93DF93D82FC92F48E050E0682F792FEF
:1027800081E0BBDF88E0ED2FFC2FA0E4B1E00190F9
:102790000D928A95E1F7DF91CF910895BC0143E056
:1027A00050E083E0AACF8F929F92AF92BF92CF92D8
:1027B000DF92EF92FF920F93CF93DF9388E090E048
:1027C0000E94FF304B015C01CAE7D3E06883998225
:1027D000AA82BB821C821D821E821F8283E290E03D
:1027E0000E94F730282F30E040E050E060E070E0D9
:1027F00080E090E000E20E943230282939294A29FD
:102800005B29288339834A835B836C837D838E8332
:102810009F83DF91CF910F91FF90EF90DF90CF904A
:10282000BF90AF909F908F9008952FB7F8948091AC
:10283000480190914901A0914A01B0914B012FBFED
:102840000895CF93DF93EC01F0DF8C1B9D0BDF919C
:10285000CF910895CF93DF93C09184038091860335
:10286000C82B809183038115F1F0DFDF20918A036B
:1028700030918B03821B930B8838934110F00E9498
:10288000AD06D091830320E08CE291E0FC01308121
:10289000019631112F5F31E082339307B9F721118F
:1028A0000E94AD06CD2BC0932A01E0916B02F091FE
:1028B0006C02309741F00280F381E02D309719F0DF
:1028C0008AE291E00995DF91CF91089510928403F7
:1028D000ECE2F1E086E0DF011D928A95E9F780E005
:1028E00090E00E94090C80E090E00E94310C109270
:1028F0008603B0CFEBDF2FEB87E299E021508040D9
:102900009040E1F700C0000088E19CE00FB6F89429
:10291000A89581BD0FBE91BDFFCFCF93C82F811564
:10292000A1F08CEF8C0F813A90F4ECE2F1E082E3BD
:1029300091E02191C21789F18E179F07D1F76C2F73
:102940008AE291E00E94590C85DFCF91089580E2E0
:102950008C0F883048F4C77081E001C0880FCA9599
:10296000EAF70E949F06F0CF8BE58C0F833038F496
:102970002C2F2452330BC9010E94090CE6CFC85AF0
:10298000CB3118F7EC2FF0E0EE0FFF1FEF50FF4FA9
:10299000808191810E94310CD8CF6C2F8AE291E026
:1029A0000E94730C57DFCBCF682F811529F18CEF74
:1029B000860F813A28F48AE291E00E94730C4ACF94
:1029C00080E2860F883048F4677081E001C0880F8C
:1029D0006A95EAF70E94A506F2CF8BE5860F833051
:1029E00020F480E090E00C94090C685A6B3120F4DC
:1029F00080E090E00C94310C08951F93CF93DF9307
:102A0000182FEB018ADF209731F4812FCDDFDF9182
:102A1000CF911F91089587EB9BE00197F1F700C0DC
:102A200000002197F0CFA0E0B0E0E9E1F5E10C94DF
:102A3000BF2FEC018881811509F1813009F045C073
:102A40008981813051F48A81239660E570E0893371
:102A500011F060E070E0D1DFEDCF823021F48A81A7
:102A600023965BDFE7CF833021F48A8123969CDFB6
:102A7000E1CF843041F022968111DCCFCDB7DEB7B3
:102A8000E9E00C94DB2F8A81239620E030E09AE085
:102A9000682F6053770BAB016A30710560F0211528
:102AA000310551F3E7EBFBE03197F1F700C000008F
:102AB00021503109F4CF929FB001939F700D1124E2
:102AC0009A01260F371F8991E3CFE82FF0E0EC57EA
:102AD000FF4FB490282F26952695269530E0F901D2
:102AE000EC58FF4FE4908770F12C082E02C0F5944B
:102AF000E7940A94E2F7E0FAEE24FF24E0F8F90103
:102B0000EC59FF4FC490D12C082E02C0D594C79425
:102B10000A94E2F7C0FACC24DD24C0F8F901EC5A9B
:102B2000FF4F049110E002C0159507958A95E2F7D2
:102B300001701127E114F10411F081EEEEDEC114F1
:102B4000D10411F086EEE9DE60E070E08B2D55DFF8
:102B5000C114D10411F086EE27DFE114F10411F065
:102B600081EE22DF0115110521F060E070E08CE2BA
:102B700044DF21965FCF811519F00E949F066ACE2F
:102B80000895811519F00E94A50664CE0895811557
:102B900031F090918603892B809386035BCE089554
:102BA000811539F08095909186038923809386035F
:102BB00051CE08958091EE02811521F082E2F0DF7E
:102BC0001092EE020895CF93DF93EC014A855B8566
:102BD0006E857F850E94F50B9B8190958091860381
:102BE0008923809386038C810E94A50633DE86E0CC
:102BF000FE0111928A95E9F7DF91CF910895CF9365
:102C0000DF93EC018D8181FD13C082608D83809103
:102C100086039B81892B809386038C810E949F066B
:102C200019DE488559856E857F85CE010E94F50B9A
:102C300010927303109272038D8180FD02C0CE0149
:102C4000C2DFDF91CF910895962F20913E0422FF9D
:102C50000FC0682F660F660F660F692B609387039E
:102C60000E94D905E2DD909389038093880308953B
:102C70000C94D90590918303292F2823211559F00D
:102C80008095892380938303811531F0CEDD809375
:102C90008A0390938B03089580E090E0F8CF6091D1
:102CA0007A036695669570E04BE050E08DE690E023
:102CB0000E94C630892B19F481E080937903B5DD39
:102CC00090932B0280932A02089590917A0390FFAB
:102CD0002CC0811559F18B3258F58F73880F880FEE
:102CE00090917A039370892B80937A03611519F080
:102CF0008AE793E0E6D960917A036695669570E07D
:102D00004BE050E08DE690E00E94C630892B91F0B8
:102D10001092790381E080932D0220E040917D03A1
:102D200060917C0380917B030DCA089581E0D6CF2A
:102D30008AE2D4CFB4DFEECF80917A038695869570
:102D40008F5F8B3208F081E061E0BFCF80917A0322
:102D5000869586958A9509F48AE261E0B6CFCF938D
:102D6000DF9380916604811571F0109266045DDD39
:102D700090930C0280930B0210921A0280911A0217
:102D8000DF91CF91089580911A028111F7CFC09100
:102D90000B02D0910C0249DD8C1B9D0B069770F342
:102DA00081E080931A02EACFA0E0B0E0EAEDF6E11C
:102DB0000C94C12F162FD72FC42FD22E811599F026
:102DC0004093760332DD9093370180933601C770CC
:102DD00081E001C0880FCA95EAF7CDDECDB7DEB736
:102DE000E7E00C94DD2F90917603491334C0E09016
:102DF0003601F090370119DD9C012E193F09790148
:102E0000812F9D2FB0D8E816F90628F5D0E2DD0D08
:102E1000CD1591F0C77011E0812F01C0880FCA95C0
:102E2000EAF7AFDED83040F48D2D877001C0110F66
:102E30008A95EAF7812F9FDE60E070E0802FDDDD6C
:102E4000D83060F62D2D277081E001C0880F2A95BB
:102E5000EAF797DEC3CFC77081E001C0880FCA953B
:102E6000EAF7F7CFA8E0B0E0E8E3F7E10C94B82F79
:102E70007C01DC0114968C91811509F4C7C161E0D5
:102E8000C7010E945C0E8C01F7018581811529F133
:102E900080917203909173030097F9F00817190756
:102EA000E1F0FC01FF27887F9927892B09F077C083
:102EB000A4E0EE0FFF1FAA95E1F7EE50FD4F8581CC
:102EC0008460858311830083CF0199DE109286038D
:102ED00061E0C7010E945C0E8C01D70115968C91B0
:102EE000811509F4ECC0C80197578038910508F0A6
:102EF00074C1003108F07AC166E670E080E090E0CD
:102F00000E94BB0E811172C1812C912C54010111C0
:102F100049C004E09E012F5F3F4F6901D601E02FB9
:102F20001D92EA95E9F724013501FFEF4F1A5F0A78
:102F30006F0A7F0AC501B4010E94BB0E8983811507
:102F400009F454C1813009F0B7C0A50194012E5F86
:102F50003F4F4F4F5F4F2D833E834F835887C301B1
:102F6000B2010E94BB0E182F8A83811509F43EC15D
:102F70008FEF810F833088F56D817E818F819885F9
:102F80000E94BB0E8B83811511F0C6014CDD24011C
:102F9000350133E0430E511C611C711C1BC0E0E085
:102FA000F0E08DCFB7E68B169104A104B10409F4CB
:102FB0001DC1C501B4010E94BB0EEFEF8E1A9E0A1F
:102FC000AE0ABE0A8111EECF0150A1CF4D805E80C6
:102FD0006F80788453014201A1CF8BEF810F833042
:102FE000A0F52401350143E0440E511C611C711C05
:102FF0006D817E818F8198850E94BB0E8B838115A8
:1030000049F3C301B2010E94BB0E8C83811108C039
:103010002401350154E0450E511C611C711CDACFAE
:103020008B819C818130AFEF9A0710F0982F882711
:10303000163029F0173031F00E945B25E9CF0E944D
:10304000F724E6CF0E942925E3CF143009F0BECF44
:103050006D817E818F8198850E94BB0E182F24017F
:103060003501B4E04B0E511C611C711CC501B4014B
:103070006D5F7F4F8F4F9F4F0E94BB0E111509F45C
:10308000B5C0811509F4B2C08150990B4FEF489F2C
:103090009001499F300D1124E12FE150FF0B2E0FBD
:1030A0003F1F2150310908F495CF87EB9BE0019732
:1030B000F1F700C00000F5CFC601B5DC8BCF0115DC
:1030C000A7E51A0708F4B5C00115B8E51B0708F015
:1030D000B8C66801E7E5DE1A64EE72E08C2D0E9446
:1030E0009E0F892B31F5C60174E0880F991F7A95E0
:1030F000E1F7FC01EE50FD4F2281213009F059C06B
:103100002091E4023091E502232B99F02091E60210
:103110003091E702232B69F02091E8023091E90217
:103120004091EA025091EB02242B352B232B09F41A
:103130004AC08091EE02811509F461C1C0908403F8
:10314000D090830372DB88579C4E9093F00280935B
:10315000EF02F7018581811509F451C18D2D8C296C
:103160008D79811120C10115F0E51F0708F0B8C065
:10317000011520E4120708F02CC1063E110509F4E0
:10318000DDC0C80190528115904208F029C1D701D5
:1031900016968C91803108F4FEC0C80199271092D0
:1031A00086038D32910509F0B4C082E080938603D6
:1031B0001BC1223009F0BDCF2091E8023091E90215
:1031C000232B09F4B6CFFC01E950FD4F20812E7F5F
:1031D00020838E509D4F13DDACCF0337FCE71F07D4
:1031E00041F58091EE028115A9F0E4DC809187031E
:1031F0008770811559F0F7018581811539F080912B
:103200003E0482FF03C082E00E9484062896E0E12B
:103210000C94D42F109284030E94AD0606DB8857CD
:103220009C4E9093F0028093EF0281E08093EE0237
:10323000DDCF023A22E51207C1F158F4C8019052DD
:103240008115904218F1013E110579F1053E1105F5
:1032500003C0023B52E5150709F06BCF25EE30E0C5
:103260002770332781E090E001C0880F2A95EAF7A4
:103270002091F1023091EE023115F9F0F70135811C
:103280003115B1F0282B2093F102B0CFD70116965B
:103290008C91803108F04DCF812F99278F7199271C
:1032A0008230910511F04297D7CF21EE30E0D8CF90
:1032B000809582238093F10299CF322F38233115E4
:1032C00009F437CF982F909592239093F1020E94A2
:1032D000A506D70115968C91811509F487CF29CFC2
:1032E000003EB2E51B0708F049C0003CE2E51E07BE
:1032F00028F5003AF2E51F07E8F4003622E5120748
:10330000E8F4C801925580349105C0F0109286030C
:10331000C8018E32910508F0B8C08832910508F0D6
:1033200061C08E31910508F05FC004974A9708F498
:103330003CCF39C0043B32E5130741F7F7019581D3
:10334000911509F49BC510927603980130572332EA
:10335000310508F07AC584E090E00E940431909332
:103360003E0480933D04F801E150F047E232F1055C
:1033700008F0DEC0EA54FE4C0C94193009374CE7D3
:10338000140728F407375CE71507C0F6BFCF0B37E3
:103390008CE71807D2CF812F8F71843179F2863173
:1033A00041F41092860306DC8091F1020E949F0690
:1033B00026C000DC8091F1020E949F06F801E851CE
:1033C000FC47E730F10508F0B9CFE852FE4C0C9409
:1033D0001930D70116968C91803108F0DECEEECFF1
:1033E000C801DDCE8A97F9F68091F102811531F09E
:1033F0008091860392E08927809386032BDAC801A7
:10340000975581159140D0F65801F8EFAF22BB24B3
:10341000A114B10409F0EACEF801FF2754E0EE0F41
:10342000FF1F5A95E1F79F012E503D4F6901D701CB
:1034300015968C91E950FD4F908180FB90F9908317
:10344000811551F1F2D99093750380937403F601BD
:1034500082818F5F82838091860390918403892B80
:103460008383809183038483468157816685778532
:10347000C6010E94F50BD60115968C9181FF58016B
:10348000B0927303A092720359CF8C34910509F462
:10349000ABCF8D329240A7CFF90144855585668523
:1034A0007785C9010E94F50BD60115968C9181FF95
:1034B00045CFC60188DB8091720390917303081792
:1034C000190709F03BCF109273031092720336CFA5
:1034D00006E221EE41EE6AE17CE7F701858108C052
:1034E00007E225EE45EE6BE17CE7D70115968C915E
:1034F0005BDC7CCE06E221EE40EE68E17CE7EDCFBE
:1035000007E225EE44EE69E17CE7EFCF06E221EE2B
:1035100042EE6CE17CE7E1CF07E225EE46EE6DE19D
:103520007CE7E3CF08E221E045EE6EE17CE7D5CF12
:1035300080913D04816080933D0460913D047091D1
:103540003E0484E090E00E943131C0D94FCE80919A
:103550003E04886080933E04F0CF80913D048260F9
:10356000EACF80913D048460E6CF80913D0488607D
:10357000E2CF80913E048160EDCF80913E04826075
:10358000E9CF80913D048061D6CF80913D04806277
:10359000D2CF80913D048064CECF98D980913D04F4
:1035A0008068C9CF80913D048C60C5CF80913E0476
:1035B0008360D0CF80913D048E7FBDCF80913E044B
:1035C000877FC8CF80913D048D7FB5CF80913D042A
:1035D0008B7FB1CF80913D04877FADCF80913E043A
:1035E0008E7FB8CF80913E048D7FB4CF80913D0413
:1035F0008F7EA1CF80913D048F7D9DCF80913D0432
:103600008F7B99CF63D980913D048F7794CF809140
:103610003D04837F90CF80913E048C7F9BCF80912F
:103620003D04992782FF939590FB82F990FB83F9E3
:1036300082CF80913E04982F909590FB80F990FB6B
:1036400081F988CF90913D04892F8F7B96FF80640C
:1036500072CF3CD990913D04892F97FB87F9805810
:103660006ACF61E08EE090E00E94183166CF60E0A2
:10367000F9CF90913D04892F8F7E94FF80615BCFBD
:1036800090913D04892F8E7F90FF816054CF90915F
:103690003E04892F877F93FF88605CCF8272F80198
:1036A000E052F847EB30F10508F055C0E152FE4C0E
:1036B0000C9419300737FCE71F0709F050C081E070
:1036C0000E94E3056EC080917A0380FF0CC08E7F5C
:1036D00080937A038AE793E00E9461101092790345
:1036E0000E94540983CD816080937A0361E08695BE
:1036F0008695EBDA7BCD811521F028DB77CD81151E
:10370000E1F31ADB73CD811529F00E941E116ECDF5
:103710008115D9F30E94161169CD811529F00E94F7
:10372000311164CD8115D9F30E9426115FCD811529
:1037300029F00E9447115ACD8115D9F30E943C11FE
:1037400055CD811529F00E94981050CD8115D9F3DF
:103750000E948E104BCD07372CE71207F9F008377F
:103760003CE7130721F19801205E324520323105F4
:1037700018F5911121C00F7181E090E0AC0102C0F9
:10378000440F551F0A95E2F78A01642F83E090E009
:103790000E941831802F0E94D30528CD81E00E941D
:1037A000D90543E062E081E00E945B061FCD82E024
:1037B000911509F485CFF3CF4091820380913C04A9
:1037C000282F30E02095309570E024233723232BD9
:1037D00019F04823409382030B375CE7150741F447
:1037E000911509F403CD0E94B0050E94CE0BFECCCA
:1037F000003482E5180708F055C00032A2E51A0728
:1038000008F057C00115B0E51B0750F50115E0E4BD
:103810001E0708F064C0911509F47AC00A35BCE7A8
:103820001B0709F4EDC008F0D1C00130FCE71F0709
:1038300009F4E4C003302CE7120709F4D9C00115DC
:103840003CE7130709F064C041D88FEB97E2A9E089
:1038500081509040A040E1F700C000000E94B111EB
:103860009801305521153240B0F6980145E0369563
:1038700027954A95E1F7822F8F702091820330E0DF
:1038800041E050E0082E02C0440F551F0A94E2F7B1
:1038900024233523232B09F4BECF9111A6CF1092F8
:1038A0008403E9C29801205C32452032310508F0DA
:1038B000B2CF802F8F712091820330E041E050E041
:1038C000082E02C0440F551F0A94E2F72423352323
:1038D000232B09F4A0CF911509F488CC86CFD7010A
:1038E00016968C91803108F096CF911111C0212F3E
:1038F0002F7081E090E002C0880F991F2A95E2F7AF
:103900002091820330E082239323892B09F06ECC2F
:10391000D70117968D919C91009709F475C00E946C
:10392000AB07D82E192FD7011596BC901597169670
:10393000AC90A2948FE0A8228091870387708115B4
:1039400009F1CB2CB114F9F0892F807F803469F014
:1039500080E28D0D8830B0F0892F807E803229F48E
:10396000B2E0DB1678F0A11469F080913E0482FF8A
:1039700009C082E00E948406809187038770CC246E
:10398000C3948111C12C812F82958F70883009F4E6
:1039900054C108F06DC0843008F04EC0012F0F7084
:1039A000823008F476C0107F103211F00295007F4B
:1039B000D11409F4A2C0F1E0DF1609F400C1B1147A
:1039C00009F40CC1A11409F4B4C076C00B354CE75E
:1039D0001407C1F080913E04002482FF0394802DDF
:1039E0000C355CE7150709F093CF0E94AC0D90CF22
:1039F0006FEF7FEF80E090E00E9431310E947A14F7
:103A000081E0F3CF80E0F1CFF7018581C080D180E4
:103A1000811569F0C6010E94330E182F682FC60168
:103A20000E94F105B601812F0E94180E78CFC601C1
:103A30000E942706182FF6CF843009F4E1C0C11484
:103A400009F42CC18091870380FD28C1D701159608
:103A50001C928695869586950E94D905C70102DA43
:103A6000809187038695869586950E94E30516C109
:103A7000893009F457C18A5F8F70823000F7E2EF16
:103A8000DE1261C1812F8F71B1105AC10E94D90518
:103A900001C1103110F00295007FB114A9F0011599
:103AA00059F080E28D0D883010F0D11007C0802FC2
:103AB0000E949F060E942A148D2D2DC0809186039E
:103AC000802B80938603F6CF8D2D0E94D414011590
:103AD00009F4B5CF80E28D0D883010F0D11004C00C
:103AE000802F0E94A50606C0009580918603802342
:103AF000809386030E942A14A2CF80913E0482FD07
:103B000014C0B11459F0011529F0802F0E949F06AE
:103B10000E942A1480E00E948D1491CF80E00E94C0
:103B2000D414011509F48BCFDBCFB11459F1A110D6
:103B300003C0802F20D883CF21E0A21211C01091A2
:103B40008303802F8123081709F479CF0E9415146D
:103B500090938B0380938A03102B109383036FCF72
:103B600035E0A3126CCF802F06D8802F83D88091A8
:103B70008503902F9823091709F461CF802B809338
:103B800085035DCFA11011C0802F0E94C115802F29
:103B900071D880918503902F9823911509F44FCF08
:103BA00000950823009385034ACF41E0A41247CF34
:103BB000809184038023811509F441CFE5CFB114AE
:103BC00029F056E0A51608F03ACFB3CF85E0A81645
:103BD00008F035CF802F0E94C11531CFA114D1F349
:103BE00099E3D91209C0AFEFBDEEE2E0A150B040B9
:103BF000E040E1F700C000008D2D0E94D4141FCFDB
:103C0000812F869586958370811569F0813009F042
:103C100016CF8D2D912F9370B11002C080E090E0EF
:103C20000E94310C0CCF8D2D912F9370B11002C0DA
:103C300080E090E00E94090C02CF812F83708111F7
:103C40003AC0B11027C04D2D429546954770440F9C
:103C5000440F8D2D8F70042E01C0880F0A94EAF74F
:103C60002D2D2071D4FE07C02FE030E001C0220FBF
:103C70004A95EAF720951695169513701230B1F013
:103C8000133091F030913B04113069F0822B832383
:103C90000E94D3050E94FA0B0E94C30560E0C70191
:103CA0000E945C0EB3CA832B822BF2CF822B9091A1
:103CB0003B048927EDCFB11451F110FFEBCF4D2D0F
:103CC000429546954770440F440F8D2D8F70042EFA
:103CD00001C0880F0A94EAF72D2D2071D4FE07C089
:103CE0002FE030E001C0220F4A95EAF720951695A3
:103CF00016951370123089F0133069F030913C043E
:103D0000113041F0822B83230E94D605C3CF82302D
:103D100008F2D5CF832B822BF7CF822B90913C04D6
:103D20008927F2CF1F70B11439F0812F0E94D90575
:103D30008D2D0E94BB15AECF8D2D0E94C115812FF8
:103D40000E94E305A7CFF3EFDF1680F420EFD21631
:103D5000E1F031EFD316A1F0B11409F460C0A11461
:103D600009F45AC08D2D0E948D1494CF43EFD416C0
:103D7000F1F054EFD512F0CF80913E0482FD23C0C4
:103D8000812F8F71B114E1F281CEB11469F085E019
:103D9000A81608F07FCF1F7181E090E0012E01C0CE
:103DA000880F0A94EAF7BACF96E0A916F2CF80E01E
:103DB000B11409F4A9CF1F7181E0012E01C0880F51
:103DC0000A94EAF7A1CFB114C1F0809187038770FC
:103DD000843049F41092870310928903109288036B
:103DE000812F8F71ADCFA5E063E0AA1608F052CF06
:103DF000812F8F710E9424164DCFB5E0AB1640F095
:103E000010928703109289031092880364E0F0CF28
:103E100081E00E9484063ECF812F8F7137CEA1149E
:103E2000F9F2E9E3DE1209C0FFEF2DEE32E0F150C6
:103E300020403040E1F700C000008D2D0E94D414D6
:103E400029CF0337FCE71F0748CA80918403063156
:103E50002CE7120709F022CC8A7A91E0811101C087
:103E600090E09093770365E3811101C069E28AE2F3
:103E700091E00E94590C0E942A14B8C906313CE70F
:103E8000130709F017CC8091770365E3811101C016
:103E900069E28AE291E00E94730CEDCFA0E0B0E00D
:103EA000E4E5FFE10C94C12F8091BD02803108F060
:103EB00049C08091BC02811509F444C0C0916E02D2
:103EC00089E0D82E80916D028C17E1F1EC2EF12C57
:103ED000DC9EE0011124FE01E159FD4F8481811532
:103EE000B1F191818091B802981331C09081809195
:103EF000B70298132CC08581811129C002811381DA
:103F00008091B9029091BA02081B190B60E087EB0F
:103F100092E00E945C0E0E94B30F08171907B8F4D4
:103F20008091BD028F7080618093BD02CB58DD4FC0
:103F300088818F708061888387EB92E00E943217BE
:103F40000E947A06CDB7DEB7E7E00C94DD2FE701DB
:103F50002196C770B7CFAFE0B0E0E1EBFFE10C9482
:103F6000B92F8C0186E0F801DE011A9601900D92BE
:103F70008A95E1F7F801F580E48087EB882E82E0EE
:103F8000982E8091BB02811117C0E11491F0F114B9
:103F900009F480C1C8010E948A0E811509F47AC112
:103FA00089E0F801A7EBB2E001900D928A95E1F764
:103FB00075DFFF24F3946AC0A280B380D090BC0266
:103FC0008091B9029091BA023501681A790AD11428
:103FD00009F411C1C080518060E087EB92E00E943B
:103FE0005C0E0E94B30F6816790608F0B6C0E114A3
:103FF00001F38091B802F8019181E090BD02F0E1F7
:10400000EF1608F064C0981320C09091B702F80131
:10401000808198131AC02091BE023091BF0287811F
:1040200090852817390789F4F1104BC08E2D8F70B9
:1040300080618093BD0287EB92E00E9432178091ED
:10404000BD02F8018683F12C21C0F1103AC040E096
:10405000652D8C2D0E94210D40E0652D8C2D0E9438
:10406000210DF82E8111EFCF8A859B850E947E0E4F
:10407000292F22952F70903470F49F702230A0F079
:104080009115B1F0F8019681903190F48F2D2F9613
:10409000EFE00C94D52F2A5F2F70223068F0C80112
:1040A0000E943217FD2CF2CF911511F0811571F39A
:1040B000805E883058F3F3CF803F40F3815F8330D8
:1040C000F9CF8091BD0281608093BD02BCCF98136F
:1040D0001EC09091B702F8018081981318C02091FA
:1040E000BE023091BF02878190852817390779F485
:1040F000F1100DC0E682C8010E94321789E0F80174
:10410000A7EBB2E001900D928A95E1F752CFC8017A
:104110000E948A0E811509F4BDC0F11409F4BAC0D9
:104120008091BD02803208F43BCF8091B70290911C
:10413000B8029A838983BC82AB828091BB028D8353
:104140001E82EF828091BE029091BF02998788877C
:10415000CE0101960E94321723CFD090BD02F0E12C
:10416000DF1650F487EB92E00E94321789E0F401E9
:1041700011928A95E9F767CFE11409F41ACF90916B
:10418000B802F801818198131AC09091B70280811A
:10419000981315C02091BE023091BF02878190858F
:1041A0002817390761F4F1100AC0D682C8010E94AD
:1041B000321789E0F40111928A95E9F7FACEC80125
:1041C0000E948A0E811509F465C0F11409F462C0D9
:1041D0008091BD02803208F4E3CE8091B7029091C5
:1041E000B8029A838983BC82AB828091BB028D83A3
:1041F0001E82DF82A7CF60E087EB92E00E945C0E18
:104200000E94B30F6816790608F0B0CFE11409F4E4
:10421000D0CEF11409F43EC09091B802F80181812A
:1042200098132EC09091B7028081981329C02091D5
:10423000BE023091BF02878190852817390701F5AA
:104240008091B9029091BA02A81AB90AF8ECAF1697
:10425000B10408F053CF8091BD0280FD4FCF803173
:1042600008F44CCFF8018683982F907F903F09F493
:1042700042CF982F907F905F8F70892B86833BCFA2
:10428000C8010E948A0E81118BCE8091BD0281608F
:104290008093BD02C8010E9432178BCEA2E1B0E02C
:1042A000E4E5F1E20C94C42F0A871B872C873D8735
:1042B0004E875F87688B798B8A8BCE010A964BDE9F
:1042C000811128C020916D0230916E0289E0FE01BB
:1042D0003A96DE01119601900D928A95E1F78E854E
:1042E0008115C1F0822F90E00196877099273817C9
:1042F0001906D9F099E0929FD0011124A159BD4F20
:10430000FE01319601900D929A95E1F780936D022E
:104310000E947A0619E080916E0290916D028913D5
:1043200012C06296E4E00C94E02F0E946614109292
:104330006D0210926E0289E0E7EBF2E0DF011D9260
:104340008A95E9F7E7CF189FC001112481599D4F45
:1043500002DE811531F380916E0290E00196877044
:10436000992780936E02D7CFEF92FF920F931F93FE
:10437000CF93DF9380913804E0915001CDE081111B
:1043800030C0CDB7DEB7E6E00C94DE2FD1E0DE0F13
:10439000D0935001EE2EF12CCE9FF0011124E0536A
:1043A000FC4F84818115E1F087819085892B21F470
:1043B00081859285019651F400811181228133819A
:1043C0004481558166817781808568DFCE9DF001CB
:1043D000CF9DF00D1124E053FC4F14821092860300
:1043E000ED2F80913804E81788F21092380410926B
:1043F0005001C7CFA4E0B0E0E0E0F2E20C94B72FA8
:104400002091CF03298397E0992E01E010E02DE061
:10441000322E34E0532E882483948091CE039981E8
:10442000891307C0A1DF0E94910B2496E1E10C944F
:10443000D32F9981892F90E09C838B83FC01EE0F11
:10444000FF1FEC53FC4F80819181989ED001999E73
:10445000B00D1124FD01E457FC4FFA83E983248158
:1044600021115BC060903804E0EDF3E060E070E0A3
:10447000712C661508F04FC0A384B484A981BA8159
:10448000CD90DC902FEF3FEF412C442D50E0760192
:10449000E40CF11CE40CF11CD701ED90FC90E1144C
:1044A000F10439F0AE14BF0409F0A90143949A0154
:1044B000ECCF2F3F3207D1F1D80102C0AA0FBB1FAA
:1044C0002A95E2F77A2A9801042C02C0220F331FA2
:1044D0000A94E2F7A901415051097416150629F50D
:1044E000369EF001379EF00D1124E053FC4F989E4C
:1044F000D001999EB00D1124A457BC4F12962D9156
:104500003C911397308727835482108211829287BF
:10451000818715968C920E94A20B8B819C810196BB
:104520009A8389838370898378CF14826F5F7F4FEA
:104530003D969FCF10923A04109239041092840055
:104540008091CE038093CF030E94910B0DCFACE1FD
:10455000B0E0EDEAF2E20C94B62F4B8B5C8B6D8BE6
:104560007E8B8F8BB92E988FA92E91111092860376
:10457000188A198A1A8A86E0FE017396DE011A9655
:1045800001900D928A95E1F75F8880913E0482FF49
:104590001FC00E9415142091880330918903821B4B
:1045A000930B8838934138F08091870382FD03C0D4
:1045B00082E00E9484060E94151420918A033091A3
:1045C0008B03821B930B8838934110F00E94AD0639
:1045D0005114D9F05E86BF8661E0CE010A960E9432
:1045E0005C0E61E0CE010A960E945C0E61E0CE0195
:1045F0000A960E945C0E4C0180356CE7960791F498
:10460000A11419F181E0809384005E86BF860A853B
:104610001B852C853D85452D5B2D688979898A8987
:104620003DDECDC081359C4721F4A11471F082DFBD
:10463000ECCF82E588168CE7980639F4A11429F0AE
:10464000809184008111F3CFDDCF4CE8E42E43E06C
:10465000F42E412C612C712CD7016D917C91CC24CE
:10466000CA94DD24DA9480E0282F30E0FB01E80FC3
:10467000F11DE80FF11D408151814115510539F0BF
:104680008416950609F096018F5F6901EDCF10E061
:10469000BFEFCB16DB0609F44EC0F7014481109141
:1046A0008400411110E0D70115963C90159716969D
:1046B0009C911697A11409F405C1111509F402C1C2
:1046C000311017C021E030E00C2C01C0220F0A94F9
:1046D000EAF7922B16969C932091CC033091CD0350
:1046E0002233310530F422E330E03093CD032093C0
:1046F000CC03E1E0F0E002C0EE0FFF1F8A95E2F785
:10470000CF010197D70116962C912817190699F415
:10471000C0903904D0903A04C114D10409F453C0B4
:104720000E9415148C199D09C39708F44CC081E0B0
:10473000F701848311E0412ABFEF6B1A7B0AE7E09F
:10474000EE0EF11CF8E06F16710409F085CFA1148C
:1047500009F417C1411409F414C10E94151490936F
:104760003A048093390480913804883040F591E010
:10477000980F9093380499E0FE013A96DE01119665
:1047800001900D929A95E1F75D82BE822DE0829FA5
:10479000C001112480539C4F29E0FE013196DC01B9
:1047A00001900D922A95E1F72FEF3FEFDC011A9669
:1047B0003C932E9319971C969C928E921B976C9605
:1047C000E2E10C94D22F2091CF038091CE03922F5F
:1047D000E0E0F0E001E0281709F448C0422F50E083
:1047E000FA01EE0FFF1FEC53FC4F2080318037E0C1
:1047F000329DF001339DF00D1124E457FC4F608190
:1048000071817C8F6B8FB0E030E0A0E0EB8DFC8D90
:10481000EA0FF11DEA0FF11DC080D180C114D1044F
:10482000E1F0F7010190F081E02DFA8FE98F30E09F
:1048300007C0E1E0C616D70609F0E0E0BE2B3F5FF7
:10484000E98DFA8DE30FF11DE30FF11D6081718198
:104850006115710571F7AF5FD9CFB11581F13A17C5
:10486000C8F4E1E0D7011496EC93F7019093CF03DD
:10487000EE15FF0509F45FCF90E0FC01EE0FFF1F7E
:10488000EC53FC4F7182608201968370992780936C
:10489000CE0351CF37E0329DF001339DF00D11244E
:1048A000E457FC4F0483EE15FF05F9F2291302C00B
:1048B0009F5F93709A012F5F3F4F23708CCFE0E092
:1048C000F0E0F8CF292F30E0311024C061E070E033
:1048D00002C0660F771F8A95E2F7CB010197281770
:1048E000390791F010E0E1E0F0E002C0EE0FFF1FA9
:1048F000CA94E2F76F01C094D70116968C9116976F
:104900008C2116968C9317CF411569F3C3010E9431
:10491000A20BE8CFA9010C2C02C0559547950A942B
:10492000E2F7C901019782239323892B39F540FFD0
:1049300025C0D70112968D919C91892BD1F087E0EB
:10494000FE013196DF011D928A95E9F70E94151448
:104950009C018B839C8384E08D83F701928183810A
:10496000792F9887898709811A8144E05E816F8158
:1049700095DCD70115961C92132DB5CF142F11700D
:10498000B2CF9091CF038091CE03981731F032DDF2
:10499000B1E04B1609F413CF38CEE6DC10923A049E
:1049A000109239040E94910BF3CFA6E0B0E0EBED3A
:1049B000F4E20C94C42F0E9415148C0180916902BA
:1049C00090916A028017910771F019821A820E94F1
:1049D0001514BC0149815A8180E090E0B8DD109344
:1049E0006A02009369022696E4E00C94E02FA6E0A8
:1049F000B0E0EDEFF4E20C94C42F8C0190936602CA
:104A000080936502011580E21807B0F4C801805E4A
:104A10009109089728F067EC75E10115110511F46B
:104A20006BEB75E1C8010E948405802F0E948D14F4
:104A30002696E4E00C94E02F80EF89838A830E941D
:104A400015148160BC0149815A8181E091E07FDDCC
:104A5000EFCFA6E0B0E0EFE2F5E20C94C42F8C01BA
:104A60009093660280936502011580E21807B0F406
:104A7000802F0E94D414C801805E9109089728F005
:104A800060ED75E10115110511F461EC75E1C801E6
:104A90000E9484052696E4E00C94E02F80EF898341
:104AA0008A830E9415148160BC0149815A8181E08A
:104AB00090E04DDDEFCFCF93DF93D82FC92F97DF55
:104AC0008D2F9C2FC6DFDF91CF9108950F931F93F9
:104AD000CF93DF938C01862F64EE72E00E949E0FCD
:104AE000892B91F4C091E402D091E502209761F006
:104AF000F8018281833039F4CE01DDDFCE01DBDFC6
:104B0000CE01D9DF01C0E0F7DF91CF911F910F9166
:104B100008950F931F93CF93DF938C01EB0164EE05
:104B200072E08C2F0E949E0F892B09F057C0FE0166
:104B3000FF27D80112968C911297EB53FE4F8130CC
:104B4000A9F415968C9182FD4EC080FF4CC082E086
:104B500080838091E6029091E7020097B9F48091FA
:104B6000E4029091E5020097C9F110C08230A1F5EE
:104B700015968C9182FD26C080FD0AC083E080835B
:104B80008091E8029091E9020097F1F030DF26C0B1
:104B900084E080838091EA029091EB020097B1F764
:104BA0008091E4029091E502009701F184DF809109
:104BB000E6029091E702009749F78091E402909114
:104BC000E502E4CF85E080838091E4029091E502E4
:104BD000009721F070DFF1CF86E08083DF91CF91E5
:104BE0001F910F91089581E08083B9CF8091E602F3
:104BF0009091E702B8CF0F931F93CF93DF938C016F
:104C0000EB0164EE72E08C2F0E949E0F892B71F4F1
:104C1000DD27CB53DE4F8881F80112821882833062
:104C2000E9F048F4813059F0823081F0DF91CF9182
:104C30001F910F9108958430B1F08530B9F78091BC
:104C4000E4029091E502009789F306C08091E602A4
:104C50009091E702009799F3FCDEE8CF8091E8029B
:104C60009091E902F7CF8091EA029091EB020097D0
:104C700099F72091E4023091E5028091E60290914B
:104C8000E70221153105F9F2009731F7C901E4CFA8
:104C9000A3E0B0E0EEE4F6E20C94BB2F8091850037
:104CA00090918600892B71F0809135018F5F809300
:104CB0003501811107C00E94490D90E09093860054
:104CC000809385003DE0C32E32E0D32EE12CF12C01
:104CD000B12C42E1A42E88248394912C6FE7762E88
:104CE000A98284010E2C01C0000F0A94EAF7102F4C
:104CF00010951A8324E630E042E050E0BE016F5F79
:104D00007F4F80E40E94E82E909386008093850078
:104D100007BB18BB09B3009510E0798224E630E0A8
:104D200041E050E0BE016F5F7F4F80E40E94302F72
:104D3000898190E0809590959695982F88279795F2
:104D4000879580789F73802B912BF601219131916B
:104D50006F018217930721F092938293BB24B3943F
:104D6000FFEFEF1AFF0A86E0E816F10409F0B8CF6A
:104D7000B11469F081E0809334010E94151490937E
:104D80003301809332012396EDE00C94D72F80916C
:104D900034018115C1F300913201109133010E9459
:104DA0001514801B910B059770F34CE050E06DE0FB
:104DB00072E085E392E00E94D330892B49F08CE0C9
:104DC000EDE0F2E0A5E3B2E001900D928A95E1F703
:104DD00010923401D8CFCDB7DEB72C970FB6F89428
:104DE000DEBF0FBECDBF84B7806884BF84B7806844
:104DF00084BF0E94151490930C0280930B0287EAE3
:104E000098E090932901809328010E946E0B0E94E4
:104E10005A0F85B7886085BF8BB780688BBF8BE4DE
:104E200080934C0480938104809358048AE5809396
:104E30004B0480938004809357048B9A8FEFA8953E
:104E4000A7EBBBE01197F1F700C000008A95B9F716
:104E50008B9878948BE083BF8BEB8CBF82E089BF0B
:104E60000E94CB0E811102C00E948C118FEF87BB74
:104E700088BB1ABA94B39B7B94BB8F988BBB85B3CA
:104E80008C6F85BB979A0E94490D90E090938600A5
:104E9000809385008CE0E5E3F2E0DF01282F1D928E
:104EA0002A95E9F7EDE0F2E0DF011D928A95E9F736
:104EB00080E090E00E940431833E9E4F21F40E94E6
:104EC000CB0E81112BC063EE7EEF80E090E00E945C
:104ED000313160E082E090E00E94183181E08093FF
:104EE0003B0461E083E090E00E94183160E074E1EF
:104EF00084E090E00E9431310E9482100E948C1167
:104F000040E050E0BA018FE090E00E94293140E09B
:104F100050E0BA0183E190E00E94293182E090E004
:104F20000E94F73080931D0284E090E00E940431DB
:104F300090933E0480933D04ABDEEFE3F9E121E082
:104F4000E150F0402040E1F700C00000A1DE809178
:104F5000350280FF08C06FEF7FEF80E090E00E9495
:104F600031310E94B11183E090E00E94F7300E943D
:104F7000D305889A9098899A91988E9A969880915C
:104F80001902811120C08AE793E00E94D313809117
:104F90007A03843030F40E9482108AE793E00E9402
:104FA000D3130E943F09109279030E94A90D8091AA
:104FB0007A0380FF05C060E0869586950E9465169D
:104FC00081E08093190288E790E090936C028093CF
:104FD0006B023FEB44ED81E0315040408040E1F70F
:104FE00000C000000E94AF16811185C00E94E91127
:104FF00080916402811509F476C180914B0484FF8D
:1050000072C146DE5EE1A52E52E0B52E65E3862E26
:1050100062E0962ED401F501219131918D919D91FF
:1050200042E0EA32F40709F49DC028173907A1F3DA
:10503000712CD4010D911D914D01F501C190D190BC
:105040005F01C016D10651F1C026D126612CEE2495
:10505000E394F12CC7018C219D21892BB1F0698249
:105060007A820E9415149C838B83F1E0FD8391E08A
:10507000970120233123232B09F490E09E8349815B
:105080005A816B817C818D8162DA6394EE0CFF1C06
:105090002FE06212DFCFF50112930293739436E092
:1050A0007312C7CF0E94840C62C080911A028115CE
:1050B000B9F080E00E94C3051092790380911C0230
:1050C00081110EC091E090931C0280917A03982F79
:1050D000917090931B028E7F80937A030E945409F3
:1050E000D7DDE5E3F2E081919191892B09F5A2E00A
:1050F000E134FA07C1F70E94AF168111D6CF0E94A2
:1051000066140E94FA0B0E94C30510921C02809143
:105110001B02811551F080917A03816080937A039C
:1051200060E0869586950E9465160E944F165ECFB8
:10513000F89491B3939A892F8C6081BB82B3BCE0C1
:105140008B2782BBEFE5FAEE20E0E150F0402040F3
:10515000E1F700C0000082B38B2782BB91BB93981C
:105160007894C9CF2817390709F062CF1EDCE09088
:105170007203F0907303E114F10439F100917403A8
:10518000109175030E941514DC01A01BB10B8D0159
:10519000C7010E94B30F80179107B8F420917203E2
:1051A00030917303C9019927287F3327232B09F0F6
:1051B000C8C024E0880F991F2A95E1F78E509D4FB3
:1051C000FC01258122FF0E94FF158091840081153A
:1051D00011F10091390410913A0401151105D9F02B
:1051E0000E941514801B910B2091CC033091CD03AC
:1051F0002817390780F49091CF038091CE03981738
:1052000009F4A2C0F7D81092CD031092CC031092EB
:105210003A04109239048091EE02811569F00E94DF
:1052200015142091EF023091F002821B930B8F3FF7
:105230009F4710F40E94DA1580917903811509F4D3
:1052400044C080917803E0917A03E695E695E81BE7
:10525000E0932C02853109F4E1C008F08CC089305C
:1052600009F4D0C008F078C0823009F4B5C08630A7
:1052700009F4BDC000ED17E099EAE92E98E0F92E97
:1052800080912D02811561F010922D020E9415145B
:1052900090932B0280932A0210922F0210922E02DA
:1052A0000E94151420912A0230912B02821B930B2D
:1052B0008F3F9F4750F4200F311F30932B022093D4
:1052C0002A028AE292E0F70109950E94FA0B182F50
:1052D00080913002181739F0109330020E94840C2C
:1052E000812F0E94C3050E94E911809164028115FB
:1052F00009F478CE8091570484FF74CE80916302C4
:10530000803209F06FCE0091670210916802E0913F
:1053100043020115110509F48CC0EE3F09F0B4C039
:1053200080914402833020F08550833008F0ACC077
:10533000E0914402EE3008F0A7C0F0E0E651FE4CE8
:1053400078C680E090E03CCF0FD810923A041092DB
:1053500039040E94910B5FCF8F3009F08BCFE69517
:10536000F0E0E459F94FE4910E2F10E0FFEFEF2E3B
:10537000F9E0FF2E85CF04EF11E05BE2E52E5BE064
:10538000F52E843209F47CCFA8F408E210E047EA55
:10539000E42E4AE0F42E883109F472CF833209F00A
:1053A00069CFE7E6F6E00591159176E8E72E79E01A
:1053B000F72E66CF853209F05DCF8E2F63E00DD6D4
:1053C000E92FF0E0EC59F94FE4910E2F10E06EEC6C
:1053D000E62E6FE0F62E54CFF0E0EB58F94FE49153
:1053E0000E2F10E083ECE82E89E0F82E49CFF0E094
:1053F000EE58F94FE4910E2F10E0B4EBEB2EB9E02C
:10540000FB2E3ECFE695F0E0E159F94FE4910E2FE7
:1054100010E0A6EDEA2EA9E0FA2E32CFF0E0E7592F
:10542000F94FE4910E2F10E0ECE5EE2EEAE0FE2EAF
:1054300027CFE43148F4E11551F0E150E33138F47D
:10544000F0E0E850FE4CF5C5EE3F09F471CF8FEF68
:105450008093430219C01092440289E08093450270
:1054600013C0809144028230A1F08330F1F081308A
:1054700071F70E94840CE3D5609345027093460255
:1054800080934702909348020E94110D109263028C
:10549000A9CD88E290E0ABD6109245021092460268
:1054A0001092470280934802EFCF80914102909181
:1054B0004202892B49F3E5E3F2E0A3E4B2E081E4A0
:1054C00092E020813181329612963C931297139686
:1054D0002C93139712968E179F0799F7D5CF80912B
:1054E0004402823009F0B3CF6091450270914602C8
:1054F0008091470290914802A2D588E290E098D628
:10550000C3CF4091460260914502809144020E94BF
:10551000E90D98278927982790934802809347029E
:10552000B3CF2091470230914802322723273227F8
:105530004091460260914502809144020E94C20D52
:10554000A3CF0E94E40EA0CF809144028238B9F12B
:10555000C0F4803809F1813809F096CF60E080917D
:1055600045020E9465169091450280917A0391113F
:105570001DC08E7F80937A03109279030E94540994
:1055800083CF833809F080CF20E040917D03609184
:1055900046028091450207C020E04091450260919B
:1055A0007C0380917B030E94A2106ECF8160809368
:1055B0007A0360E0869586950E94651665CF809196
:1055C000450280937E0360CF809144028238F1F0DF
:1055D00060F48038B1F0813809F056CF80917A03B9
:1055E00080FF12C08695869539CF833809F04CCF5D
:1055F00080917B038093450280917C0380934602D7
:1056000043CF80917D032ACF80E028CF80917E0315
:1056100025CF0E943F098AE793E00E94611034CFB2
:1056200080E18093440230CF1092440287E616CF87
:10563000009146020D3108F027CF809044029090EF
:105640004502982489249824A12CB12C33E4E32E1C
:1056500032E0F32E10E00D5B1D4FE016F10609F469
:1056600013CF80E0F7E68F169104A104B10420F473
:10567000C40187569C4FBBD5D70114968C93BFEFBE
:10568000EB1AFB0AEFEF8E1A9E0AAE0ABE0AE5CFAE
:105690008091410290914202892B09F4F5CE8091CC
:1056A00046028D3108F0F0CE882E912CA12CB12C21
:1056B000C0904402D0904502DC24CD24DC24E12CAF
:1056C000F12C03E412E0412C512C3201481459040E
:1056D0006A047B0408F0D8CEF7E6CF16D104E104C3
:1056E000F10438F4D80114966C91C60187569C4F8A
:1056F0009FD5BFEF4B1A5B0A6B0A7B0AEFEFCE1AFE
:10570000DE0AEE0AFE0A0F5F1F4FE0CF0E94521121
:10571000BBCE84E086CF809146028D3108F0B4CEB6
:10572000882E912CA12CB12CC0904402D09045021F
:10573000DC24CD24DC24E12CF12C412C512C320131
:1057400007E412E0481459046A047B0408F09CCE74
:1057500080E0F0EDCF16F2E0DF06E104F10418F48A
:10576000C601899644D5D8018D938D01BFEF4B1AA0
:105770005B0A6B0A7B0AEFEFCE1ADE0AEE0AFE0A1C
:10578000E1CF20914602022F10E02D3108F07CCEAF
:1057900080914402909145029827892798272C01EF
:1057A000612C712C803DF2E09F0708F06DCE822EB7
:1057B000912CA12CB12C40ED52E060E070E0441936
:1057C000550966097709421751056105710508F405
:1057D0005BCE2091410230914202232B29F103E458
:1057E00012E0C12CD12C7601C814D904EA04FB04C0
:1057F00008F04ACE40ED441642E0540661047104BC
:1058000030F4D80114966C91C201899611D5BFEF7E
:10581000CB1ADB0AEB0AFB0AEFEF4E1A5E0A6E0A9E
:105820007E0A0F5F1F4FE0CF6C0129E2C20ED11C30
:1058300080FBEE24FF24E0F880FF0DC08896D7D4CB
:105840009091470289279827892781159C4719F449
:105850008FEF80934702D501C401840D951DA61DCD
:10586000B71D80FF16C0C80101979C878B87D801A0
:10587000AA5BBD4F1D01C601800F911FB8D4F10175
:10588000908181159C4719F48FEFD1018C930B8582
:105890001C85F701ED5BFD4F2FEFE016F10608F0D8
:1058A0009ECF9481858181159C4711F424832583A3
:1058B00032E0E30EF11C3296F0CF809141029091DC
:1058C0004202892B09F4E0CD0E94110DFFE729EA7D
:1058D00033E0F15020403040E1F700C0000041CB00
:1058E00088E0E7E8F0E0DE01119601900D928A95DC
:1058F000E1F7E4E4F2E08FE1DF011D928A95E9F738
:1059000086E08093430288E0FE013196A7E4B2E08E
:1059100001900D928A95E1F7B7CD8CE68093430212
:1059200081E0809344021092450210924602ACCD71
:105930008091450290914602092E000CAA0BBB0BE8
:1059400025E0880F991FAA1FBB1F2A95D1F7AC012C
:10595000BD01405E5F4F6F4F7F4F481759076A0781
:105960007B0708F491CD8C36E1E09E07A105B105D7
:1059700008F08ACD4D36F1E05F076105710520F032
:105980004CE651E060E070E0481B590BBC016758E1
:10599000794F83E492E0F1D377CD4AE150E06FEFA5
:1059A00070E089E492E00CD480914102809343023C
:1059B0000093440285E0809345021092460284E001
:1059C000809347028DE06ECD81E090E09093680275
:1059D0008093670282E390E09093340280933302D5
:1059E0000E94151490933202809331024DCD01151F
:1059F000110581F1F0903F02E0903E02C09031022B
:105A0000D09032020E9415148C199D09853691059B
:105A100050F1E5FE28C0F0FE26C00E9415149093B8
:105A200032028093310280913302909134020197C7
:105A30009093340280933302892B61F410926802B0
:105A40001092670281E090E09093420280934102BD
:105A500000E010E0809141028093430200934402F1
:105A600080913302FBCC82E390E0909334028093E8
:105A70003302F0CF109242021092410205CD40E273
:105A800050E06FEF70E083E492E09AD3FDCC809118
:105A90004502823009F457C090F481113BC0E5E41F
:105AA000F2E08DE1DF011D928A95E9F788E08093AD
:105AB00043028093440283E080936202E5CC83300A
:105AC00009F478C0843009F0DFCC109146028AE0F6
:105AD000E7E4F2E0DE01119601900D928A95E1F77C
:105AE00089859A850E94610B9A8789878FEF183084
:105AF00060F4FAE01F9FB0011124675B7C4F4AE01D
:105B000050E0CE010196B1D380E0809343020E9421
:105B10005A0FBACC809146029AE0F92E8E010F5F9F
:105B20001F4FF8012F2D11922A95E9F7B8010E9415
:105B30009E0F80934302F801A4E4B2E001900D921D
:105B4000FA94E1F7A1CC109146028AE0E7E4F2E092
:105B5000DE01119601900D928A95E1F789819A8173
:105B60000E94610B9A8389838B819C810E94610BC7
:105B70009C838B838D819E810E94610B9E838D838C
:105B80008F8198850E94610B98878F838FEF1830E3
:105B900060F43AE0139FB001112467507D4F4AE052
:105BA00050E0CE01019661D380E0809343020E94D1
:105BB0006E0B6ACC209146026AE0CE010196DC01B0
:105BC000E62F1D92EA95E9F78C01283080F4629F58
:105BD000B0011124675B7C4F4AE050E0F8D280E0CE
:105BE000809343028AE0F801A4E4B2E091CE8FEF03
:105BF000F7CF78941F921FB61F9211248F939F9313
:105C0000AF93BF938091480190914901A0914A01BF
:105C1000B0914B010196A11DB11D80934801909355
:105C20004901A0934A01B0934B01BF91AF919F915D
:105C30008F911F901FBE1F901895FF920F931F9377
:105C4000CF93DF93182FEB0116BE84EA86BF0E9424
:105C50001514082FF92E06B607FE22C081B1887FE1
:105C6000883021F081B1887F803179F513B984E8DB
:105C700086BF0E941514182F092F06B607FE1DC0F7
:105C800021B1287F80E090E0283199F081E090E018
:105C9000203411F480E090E091958195910909C03C
:105CA000802F9F2D0E942114C817D907A0F68EEFD0
:105CB0009FEFCDB7DEB7E5E082C1812F902F0E9424
:105CC0002114C817D907C8F6F2CF8FEF9FEFF1CF95
:105CD00011B887E080B985B3836085BB86B78460DF
:105CE00086BF86B7816086BF86B7806486BF089509
:105CF0000F931F93CF93DF93EB0183B984E886BFA3
:105D00000E941514182F092F06B607FE10C021B1E6
:105D1000287F81E090E0283211F480E090E09195B6
:105D200081959109DF91CF911F910F910895CF3FF8
:105D3000DC0751F3812F902F0E942114C817D90737
:105D400018F78EEF9FEFEECF0F931F93CF93DF9354
:105D5000EC0184EC86BF0E941514182F092F06B69B
:105D600007FE07C083B190E0DF91CF911F910F91A3
:105D70000895CF3FDC0799F3812F902F0E942114C3
:105D8000C817D90760F78EEF9FEFEECF0F931F93E1
:105D9000CF93DF93EC0184E886BF0E941514182F7F
:105DA000092F06B607FE07C083B190E0DF91CF91BF
:105DB0001F910F910895CF3FDC0799F3812F902F0A
:105DC0000E942114C817D90760F78EEF9FEFEECF1E
:105DD000A0E0B0E0EDEEFEE2CEC0782EB62EA72E0B
:105DE0006A0189010E9415144C010431110500F16A
:105DF0000F3F100709F1C80164E170E0A3D0F62E4F
:105E0000E72E6F2D7E2D872D18DFEC01892BB9F43D
:105E1000EB2CFA2CCE0CDF1CEC14FD0411F02097B7
:105E2000C1F084E986BFCE01CDB7DEB7EDE0BFC0DB
:105E3000FF24F394E12CE5CF85E0F82EFBCF0F3F54
:105E40001007F9F2C4010E94211408171907C8F6B7
:105E5000DFCFB801F70181917F014ADFEC01DCCF90
:105E6000A3E0B0E0E5E3FFE287C07B016A018901BE
:105E7000816089830E9415144C010431110558F189
:105E80000F3F100761F1C80164E170E05BD0B62EEE
:105E9000A72E6B2D7A2D8981D0DE8A839B83EA81A0
:105EA000FB81EF2BF9F4A12CB12CF1E0CF1AD10832
:105EB000AC14BD0488F5EA81FB81F7FF1DC084E9BD
:105EC00086BF8A819B811816190614F480E090E041
:105ED0002396ECE06DC0BB24B394A12CDACF85E00F
:105EE000B82EFBCF0F3F1007A1F2C4010E9421146E
:105EF0000817190770F6D7CFC80126DF8A839B835E
:105F0000EA81FB81F7FD04C0F701EA0DFB1D8083E8
:105F10009FEFA91AB90ACCCF8A819B8197FDCFCF79
:105F2000C80134DF8A839B83EA81FB81F7FD05C0CA
:105F3000EC0CFD1CF7018083C2CFEEEFFFEFFB837B
:105F4000EA83BDCFAA1BBB1B51E107C0AA1FBB1F21
:105F5000A617B70710F0A61BB70B881F991F5A95F5
:105F6000A9F780959095BC01CD0108952F923F929D
:105F70004F925F926F927F928F929F92AF92BF9259
:105F8000CF92DF92EF92FF920F931F93CF93DF9305
:105F9000CDB7DEB7CA1BDB0B0FB6F894DEBF0FBE62
:105FA000CDBF09942A88398848885F846E847D84AF
:105FB0008C849B84AA84B984C884DF80EE80FD80B1
:105FC0000C811B81AA81B981CE0FD11D0FB6F89427
:105FD000DEBF0FBECDBFED010895992778E0880F91
:105FE000991F961708F0961B881F7A95C9F7809518
:105FF000089587FB082E062687FD819567FD61952C
:10600000ECDF0EF4919507FC8195089597FB072E20
:1060100016F4009406D077FD08D094DF07FC05D075
:106020003EF4909581959F4F0895709561957F4FAF
:106030000895EE0FFF1F0590F491E02D0994692754
:1060400096276927782787277827089572D13323E1
:1060500012F48A1B9B0B01C06CD1B7FF0895821B01
:10606000930B0895002E083090F0982F872F762FED
:10607000652F542F432F322F22270850F4CF220FA1
:10608000331F441F551F661F771F881F991F0A95CE
:10609000B2F7002D089597FD1094002E083098F067
:1060A0000850232F342F452F562F672F782F892FF5
:1060B000912DF4CF1594979587957795679557957A
:1060C0004795379527950A95AAF71124002D08952D
:1060D0008F929F92AF92BF92CF92DF92EF92FF92F8
:1060E000CF93DF93EC01688179818A819B8161156F
:1060F00071058105910521F464E279ED8BE597E066
:106100002DE133EF41E050E0C6D049015A019B0137
:10611000AC01A7EAB1E4DBD06B017C01ACEEB4EFDB
:10612000A5019401E0D0DC01CB018C0D9D1DAE1DBD
:10613000BF1DB7FF03C00197A109B04888839983A9
:10614000AA83BB839F77DF91CF91FF90EF90DF9081
:10615000CF90BF90AF909F908F900895B9CF80E679
:1061600090E0B6CFA0E0B0E0809360009093610033
:10617000A0936200B09363000895FB01DC0102C0AC
:1061800005900D9241505040D8F70895FC014150C0
:10619000504030F001900616D1F73197CF010895A5
:1061A000882799270895FB01DC0104C08D91019097
:1061B000801921F441505040C8F7881B990B08956D
:1061C000DC0101C06D9341505040E0F70895DC01BF
:1061D000CB01FC01E199FECF06C0FFBBEEBBE09A0C
:1061E00031960DB20D9241505040B8F70895E199A3
:1061F000FECF9FBB8EBBE09A99278DB30895A6E191
:10620000B0E044E050E0E5CFA8E1B0E042E050E08B
:10621000E0CFDC01A40FB51F4150504040F0CB014E
:10622000840F951F2E9105D041505040D8F7089506
:10623000262FE199FECF9FBB8EBBE09A01970DB24E
:10624000021631F02DBB0FB6F894E29AE19A0FBE18
:1062500008950396272FEDDFEBDF252FEADF242FAC
:10626000E8CF0196272FE5DFE3CFDC01CB0102C0A9
:106270002D9105D041505040D8F70895262FE1992F
:10628000FECF9FBB8EBB2DBB0FB6F894E29AE19A6E
:106290000FBE01960895052E97FB16F400940FD0BB
:1062A00057FD05D024D007FC02D046F408C0509515
:1062B0004095309521953F4F4F4F5F4F08959095F2
:1062C0008095709561957F4F8F4F9F4F089531D086
:1062D000A59F900DB49F900DA49F800D911D11243A
:1062E0000895B7FFF4CFF3DF821B930B0895A1E26B
:1062F0001A2EAA1BBB1BFD010DC0AA1FBB1FEE1F40
:10630000FF1FA217B307E407F50720F0A21BB30B8A
:10631000E40BF50B661F771F881F991F1A9469F706
:1063200060957095809590959B01AC01BD01CF0162
:106330000895A29FB001B39FC001A39F700D811D5E
:106340001124911DB29F700D811D1124911D08957E
:10635000F894FFCFEF12FB12FB12FB12FB12F912A3
:10636000FE12FB12EB1211131C131413DA1A401B4A
:10637000E21AAD1AB11AE61AB51AEA1AF61AC11AD1
:10638000391BC51AFA1AC91AFE1A221BCD1A021B8A
:10639000291BD21A071B0F1BB91AEE1ABD1AF21AC3
:1063A000D61A0B1B191B311B371BA71ADE1A471BEA
:1063B0007A1A801A681A701A861A8C1A921A631B33
:1063C0007B1B7F1B831B881B8D1B921B971B9C1B9E
:1063D000A11BA61B702C8D2C982C442A442ACD2C52
:1063E000E42CF72C3A2D3F2D442A442A442A472DE9
:1063F0002B2A312A6F2A812A912AA12AA42AE42A47
:10640000092B272A5D2C102B142B182B482B862B9D
:06641000892B8B2BC12B30
:1064160001000000FF5A0000010001010201191AE3
:106426001B1C1D1E1F202122810CB813900C910CE1
:10643600CE13AF1301FFFFF7205EE38E8D0FC90069
:106446000001020202020606060909090909090FE6
:106456000F0F0F0F0F1515151819191919191919E5
:106466001919192324252525252525E200E900EA01
:1064760000B500B600B700CD008301CC008A0192BA
:106486000194012102230224022502260227022A60
:1064960002B300B4006F0070009F01CB019F02A001
:1064A60002E200E900EA00B500B600B700CD0083BD
:1064B60001CC008A019201940121022302240225C3
:1064C60002260227022A02B300B4006F0070009F62
:0864D60001CB019F02A00200AE
:00000001FF
